:040000000200673261
:01000B0032C2
:0100130032BA
:01001B0032B2
:20002300322B2B2B204D4944492056656C6F63697479204368616E67657220312E31202F81
:2000430020415438394332303531202F202843292053746F6666656C2030342F32303037FA
:20006300202B2B2B758121C2D3C2D4758920758840758DFF75987C75A800752000C298C2E7
:20008300993098FDC298859908E508B4FE053092F0803E54F8B4F8028037E508B49006D2B1
:2000A30000C201802C30E704C20080252000028020200104D2018019E5086013209305756C
:1B00C3000860800B209405750840800375087FC2018508993099FDC29980A60A
:00000001FF
